:100000000C945D000C9485000C9485000C94850084
:100010000C9485000C9485000C9485000C9485004C
:100020000C9485000C9485000C9485000C9485003C
:100030000C9485000C9485000C9485000C9485002C
:100040000C94FE170C9485000C946E180C944818B0
:100050000C9485000C9485000C9485000C9485000C
:100060000C9485000C94850000000008000201003B
:100070000003040700000000000000000000000072
:10008000250028002B0000000000240027002A0083
:10009000040404040404040402020202020203032E
:1000A0000303030301020408102040800102040836
:1000B0001020010204081020A01811241FBECFEF49
:1000C000D8E0DEBFCDBF12E0A0E0B1E0E8EBFEE398
:1000D00002C005900D92AE33B107D9F722E0AEE32E
:1000E000B2E001C01D92A93FB207E1F710E0CDE5F3
:1000F000D0E004C02197FE010E94271ECC35D10715
:10010000C9F70E94D9180C945A1F0C940000EF9262
:10011000FF920F931F93CF93DF938B01EA01E88146
:10012000F981E284F384DB01ED91FC910680F78193
:10013000E02D61E070E0C8010995482F61E070E0B2
:10014000CE01F7010995E881F981E484F584D801AD
:10015000ED91FC910084F185E02D61E070E0C80133
:100160000995482F61E070E0CE01F7010995E8811B
:10017000F981E284F384D801ED91FC910680F78146
:10018000E02D62E070E0C8010995482F62E070E060
:10019000CE01F7010995E881F981E484F584D8015D
:1001A000ED91FC910084F185E02D62E070E0C801E2
:1001B0000995482F62E070E0CE01F7010995E881CA
:1001C000F981E688F788D801ED91FC910284F385E6
:1001D000E02D64E070E0C8010995482F64E070E00C
:1001E000CE01F7010995E881F981E688F788D80101
:1001F000ED91FC910284F385E02D6CE070E0C80184
:100200000995482F6CE070E0CE01F7010995E8816F
:10021000F981E688F788D801ED91FC910284F38595
:10022000E02D63E070E0C8010995482F61E070E0BF
:10023000CE01F7010995E881F981E688F788D801B0
:10024000ED91FC910284F385E02D61E070E0C8013E
:100250000995482F62E070E0CE01F7010995E88129
:10026000F981E688F788D801ED91FC910284F38545
:10027000E02D62E070E0C8010995482F63E070E06E
:10028000CE01F7010995E881F981E688F788D80160
:10029000ED91FC910284F385E02D60E070E0C801EF
:1002A0000995482F60E070E0CE01F7010995E881DB
:1002B000F981E688F788D801ED91FC910284F385F5
:1002C000E02D6DE070E0C8010995482F6DE070E009
:1002D000CE01F7010995E881F981E688F788D80110
:1002E000ED91FC910284F385E02D6EE070E0C80191
:1002F0000995482F6EE070E0CE01F7010995E8817D
:10030000F981E688F788D801ED91FC910284F385A4
:10031000E02D6BE070E0C8010995482F6BE070E0BC
:10032000CE01F7010995E881F981E688F788D801BF
:10033000ED91FC910284F385E02D6AE070E0C80144
:100340000995482F6AE070E0CE01F7010995E88130
:10035000F981E688F788D801ED91FC910284F38554
:10036000E02D68E070E0C8010995482F68E070E072
:10037000CE01F7010995E881F981E688F788D8016F
:10038000ED91FC910284F385E02D69E070E0C801F5
:100390000995482F69E070E0CE01F701DF91CF9118
:1003A0001F910F91FF90EF900994EF92FF920F939E
:1003B0001F93CF93DF938B01EA01E881F981E284F7
:1003C000F384DB01ED91FC910680F781E02D61E083
:1003D00070E0C8010995482F61E070E0CE01F70197
:1003E0000995E881F981E484F584D801ED91FC91C7
:1003F0000084F185E02D61E070E0C8010995482F87
:1004000061E070E0CE01F7010995E881F981E284AD
:10041000F384D801ED91FC910680F781E02D62E034
:1004200070E0C8010995482F62E070E0CE01F70145
:100430000995E881F981E484F584D801ED91FC9176
:100440000084F185E02D62E070E0C8010995482F35
:1004500062E070E0CE01F7010995E881F981E68854
:10046000F788D801ED91FC910284F385E02D64E0DA
:1004700070E0C8010995482F64E070E0CE01F701F3
:100480000995E881F981E688F788D801ED91FC911A
:100490000284F385E02D6CE070E0C8010995482FD7
:1004A0006CE070E0CE01F7010995E881F981E688FA
:1004B000F788D801ED91FC910284F385E02D60E08E
:1004C00070E0C8010995482F61E070E0CE01F701A6
:1004D0000995E881F981E688F788D801ED91FC91CA
:1004E0000284F385E02D63E070E0C8010995482F90
:1004F00062E070E0CE01F7010995E881F981E688B4
:10050000F788D801ED91FC910284F385E02D61E03C
:1005100070E0C8010995482F63E070E0CE01F70153
:100520000995E881F981E688F788D801ED91FC9179
:100530000284F385E02D62E070E0C8010995482F40
:1005400060E070E0CE01F7010995E881F981E68865
:10055000F788D801ED91FC910284F385E02D6DE0E0
:1005600070E0C8010995482F6DE070E0CE01F701F9
:100570000995E881F981E688F788D801ED91FC9129
:100580000284F385E02D6EE070E0C8010995482FE4
:100590006EE070E0CE01F7010995E881F981E68807
:1005A000F788D801ED91FC910284F385E02D6BE092
:1005B00070E0C8010995482F6BE070E0CE01F701AB
:1005C0000995E881F981E688F788D801ED91FC91D9
:1005D0000284F385E02D6AE070E0C8010995482F98
:1005E0006AE070E0CE01F7010995E881F981E688BB
:1005F000F788D801ED91FC910284F385E02D68E045
:1006000070E0C8010995482F68E070E0CE01F7015D
:100610000995E881F981E688F788D801ED91FC9188
:100620000284F385E02D69E070E0C8010995482F48
:1006300069E070E0CE01F701DF91CF911F910F913A
:10064000FF90EF900994EF92FF920F931F93CF9337
:10065000DF938B01EA01E881F981E284F384DB0115
:10066000ED91FC910680F781E02D61E070E0C8011A
:100670000995482F61E070E0CE01F7010995E88106
:10068000F981E484F584D801ED91FC910084F18531
:10069000E02D61E070E0C8010995482F61E070E04D
:1006A000CE01F7010995E881F981E284F384D8014C
:1006B000ED91FC910680F781E02D62E070E0C801C9
:1006C0000995482F62E070E0CE01F7010995E881B5
:1006D000F981E484F584D801ED91FC910084F185E1
:1006E000E02D62E070E0C8010995482F62E070E0FB
:1006F000CE01F7010995E881F981E688F788D801EC
:10070000ED91FC910284F385E02D64E070E0C80176
:100710000995482F64E070E0CE01F7010995E88162
:10072000F981E688F788D801ED91FC910284F38580
:10073000E02D6CE070E0C8010995482F6CE070E096
:10074000CE01F7010995E881F981E688F788D8019B
:10075000ED91FC910284F385E02D61E070E0C80129
:100760000995482F61E070E0CE01F7010995E88115
:10077000F981E688F788D801ED91FC910284F38530
:10078000E02D62E070E0C8010995482F62E070E05A
:10079000CE01F7010995E881F981E688F788D8014B
:1007A000ED91FC910284F385E02D63E070E0C801D7
:1007B0000995482F63E070E0CE01F7010995E881C3
:1007C000F981E688F788D801ED91FC910284F385E0
:1007D000E02D60E070E0C8010995482F60E070E00E
:1007E000CE01F7010995E881F981E688F788D801FB
:1007F000ED91FC910284F385E02D6DE070E0C8017D
:100800000995482F6DE070E0CE01F7010995E88168
:10081000F981E688F788D801ED91FC910284F3858F
:10082000E02D6EE070E0C8010995482F6EE070E0A1
:10083000CE01F7010995E881F981E688F788D801AA
:10084000ED91FC910284F385E02D6BE070E0C8012E
:100850000995482F6BE070E0CE01F7010995E8811A
:10086000F981E688F788D801ED91FC910284F3853F
:10087000E02D6AE070E0C8010995482F6AE070E059
:10088000CE01F7010995E881F981E688F788D8015A
:10089000ED91FC910284F385E02D68E070E0C801E1
:1008A0000995482F68E070E0CE01F7010995E881CD
:1008B000F981E688F788D801ED91FC910284F385EF
:1008C000E02D69E070E0C8010995482F69E070E00B
:1008D000CE01F701DF91CF911F910F91FF90EF9023
:1008E0000994EF92FF920F931F93CF93DF938B01A5
:1008F000EA01E881F981E284F384DB01ED91FC9166
:100900000680F781E02D60E070E0C8010995482F6E
:1009100060E070E0CE01F7010995E881F981E48497
:10092000F584D801ED91FC910084F185E02D60E023
:1009300070E0C8010995482F60E070E0CE01F70132
:10094000DF91CF911F910F91FF90EF9009944F92FB
:100950005F926F927F92AF92BF92CF92DF92EF92AF
:10096000FF920F931F93CF93DF93EB018A01DA017C
:10097000ED91FC91E284F384E881F9810680F781AE
:10098000E02D61E070E0CE010995482F61E070E054
:10099000C801F7010995D801ED91FC91E484F58433
:1009A000E881F9810084F185E02D61E070E0CE01FD
:1009B0000995482F61E070E0C801F7010995E881C9
:1009C000F9810680F781E02D62E070E0CE010995A3
:1009D000682F880F770B60587F4F072E000C880B0D
:1009E000990B0E94DD1C20E030E045E553E40E94B5
:1009F000921D20E030E044E752E40E94331C6B017A
:100A00007C01E881F9810084F185E02D62E070E0ED
:100A1000CE010995682F880F770B60587F4F072EFE
:100A2000000C880B990B0E94DD1C20E030E045E5AE
:100A300053E40E94921D20E030E044E752E40E941B
:100A4000331C2B013C01D801ED91FC91A284B384AD
:100A500020E030E04FE753E4C701B6010E948D1D4E
:100A6000181664F020E030E040E053E4C701B6011E
:100A70000E94C11B0E94A51C462F01C04FE762E0E7
:100A800070E0C801F5010995D801ED91FC91E4846D
:100A9000F58420E030E04FE753E4C301B2010E9447
:100AA0008D1D181664F020E030E040E053E4C301EF
:100AB000B2010E94C11B0E94A51C462F01C04FE736
:100AC00062E070E0C801F7010995D801ED91FC9151
:100AD000E688F788E881F9810284F385E02D64E0F7
:100AE00070E0CE010995482F64E070E0C801F7017D
:100AF0000995D801ED91FC91E688F788E881F981A4
:100B00000284F385E02D6CE070E0CE010995482F5A
:100B10006CE070E0C801F7010995D801ED91FC91F6
:100B2000E688F788E881F9810284F385E02D61E0A9
:100B300070E0CE010995482F61E070E0C801F7012F
:100B40000995D801ED91FC91E688F788E881F98153
:100B50000284F385E02D62E070E0CE010995482F14
:100B600062E070E0C801F7010995D801ED91FC91B0
:100B7000E688F788E881F9810284F385E02D63E057
:100B800070E0CE010995482F63E070E0C801F701DD
:100B90000995D801ED91FC91E688F788E881F98103
:100BA0000284F385E02D60E070E0CE010995482FC6
:100BB00060E070E0C801F7010995D801ED91FC9162
:100BC000E688F788E881F9810084F185E02D62E00C
:100BD00070E0CE010995D82EE881F9810284F38571
:100BE000E02D6DE070E0CE01099541E0BDEBDB1634
:100BF0000CF440E0482B6DE070E0C801F701099566
:100C0000D801ED91FC91E688F788E881F9810680AA
:100C1000F781E02D62E070E0CE010995D82EE881E1
:100C2000F9810284F385E02D6EE070E0CE01099534
:100C300041E0BDEBDB160CF440E0482B6EE070E0C9
:100C4000C801F7010995D801ED91FC91E688F78874
:100C5000E881F9810284F385E02D6BE070E0CE013C
:100C60000995482F6BE070E0C801F7010995D8019C
:100C7000ED91FC91E688F788E881F9810284F3859B
:100C8000E02D6AE070E0CE010995482F6AE070E03F
:100C9000C801F7010995D801ED91FC91E688F78824
:100CA000E881F9810284F385E02D68E070E0CE01EF
:100CB0000995482F68E070E0C801F7010995D8014F
:100CC000ED91FC91E688F788E881F9810284F3854B
:100CD000E02D69E070E0CE010995482F69E070E0F1
:100CE000C801F701DF91CF911F910F91FF90EF9015
:100CF000DF90CF90BF90AF907F906F905F904F90BC
:100D000009940F931F93CF938C01C62F0E94AB1BA6
:100D1000C81721F06C2FC8010E94B31B8C2FCF91F4
:100D20001F910F910895FC01918D228D892F90E0E4
:100D3000805C9F4F821B91098F739927089580E0F3
:100D400090E0892B29F00E94601781110C9400001B
:100D50000895DC01ED91FC910284F385E02D6DE0B6
:100D600070E00994FC0197859F7121F490899F7729
:100D700081E009F080E00895FC0197859F719D3026
:100D800029F490899F7781E0903509F080E00895FB
:100D90009B0177FF02C0295F3F4F43E035952795C0
:100DA0004A95E1F7FC01E20FF31F278530E0CB0104
:100DB00068E070E00E94FF1DA90102C055954795AB
:100DC0008A95E2F7CA0181700895660F771F860F32
:100DD000971FFC01828980580895660F771F860F40
:100DE000971FFC01818980580895FC0114A608957D
:100DF000FC0184A50895860F971F4195FC0141874A
:100E00000895860F971FFC01418708959B01442395
:100E1000E9F077FF02C0295F3F4F53E035952795F2
:100E20005A95E1F7FC01E20FF31FCB0168E070E097
:100E30000E94FF1D21E030E0A90102C0440F551FB0
:100E40008A95E2F7CA019381892B1DC077FF02C002
:100E5000295F3F4F43E0359527954A95E1F7FC011F
:100E6000E20FF31FCB0168E070E00E94FF1D21E05C
:100E700030E0A90102C0440F551F8A95E2F7CA016C
:100E800080959381892383830895660F771FFC01E2
:100E9000E60FF71F8FE7489F402D112440584683E7
:100EA00008956F5F7F4F660F771FFC01E60FF71FF6
:100EB0008FE7489F402D1124405843830895660FC3
:100EC000771F860F971F4058FC01468308956F5F78
:100ED0007F4F660F771F860F971F4058FC01438393
:100EE0000895FC01138280E8848385838683878349
:100EF0008087118612860895CF92DF92EF92FF923B
:100F00000F931F93CF93DF938C01EB017A01DC01E8
:100F100015968D919C9116978130910521F002973D
:100F200009F45DC014C0E881F9810088F189E02DE1
:100F3000CB010995882331F082E090E0F801968397
:100F40008583C3C1D80116961C921E921597D701AE
:100F5000ED91FC91C284D384E881F9810680F78108
:100F6000E02D60E070E0CE010995682F880F770BC7
:100F7000880B990B0E94DD1CAB01BC01C8010E94CB
:100F80008A11482F60E070E0C701F6010995D7018A
:100F9000ED91FC91C484D584E881F9810084F185C8
:100FA000E02D60E070E0CE010995682F880F770B87
:100FB000880B990B0E94DD1CAB01BC01C8010E948B
:100FC0008A11482F60E070E0C701F601DF91CF91F0
:100FD0001F910F91FF90EF90DF90CF900994D8016F
:100FE0001396ED91FC9114973496EE0FFF1FE00FCE
:100FF000F11F4081518157FF02C04F5F5F4F5595F0
:101000004795D701ED91FC910284F385E02D60E0D6
:1010100070E0C7010995D8011396ED91FC911497E2
:101020003896EE0FFF1FE00FF11F4081518157FFEF
:1010300002C04F5F5F4F55954795D701ED91FC91E9
:101040000484F585E02D60E070E0C7010995E88132
:10105000F9810088F189E02DCE010995882309F4F2
:101060004DC1F8018781E881F9810284F385E02D83
:10107000882309F461C062E070E0CE010995811116
:1010800074C1E881F9810284F385E02D63E070E0AA
:10109000CE010995811169C1E881F9810284F38546
:1010A000E02D61E070E0CE01099581115EC1E8811B
:1010B000F9810284F385E02D60E070E0CE010995AE
:1010C000811153C1E881F9810284F385E02D68E044
:1010D00070E0CE010995811148C1E881F98102844F
:1010E000F385E02D69E070E0CE01099581113DC1E5
:1010F000E881F9810284F385E02D6AE070E0CE0199
:101100000995811132C1E881F9810284F385E02DCE
:101110006BE070E0CE010995811127C1E881F9816A
:101120000284F385E02D64E070E0CE010995811121
:101130001CC1F801178219C163E070E0CE01099566
:101140008823C1F0D8011396ED91FC911497EE0F0E
:10115000FF1FE00FF11F808591858230910514F00B
:10116000019702C081E090E09187808781E0F801DB
:101170008783FBC0E881F9810284F385E02D62E07A
:1011800070E0CE0109958823A1F0D8011396ED9166
:10119000FC911497EE0FFF1FE00FF11F20853185A2
:1011A00080899189019728173907F4F6C9010196BA
:1011B000DBCFE881F9810284F385E02D61E070E006
:1011C000CE0109958823A1F0D8011396ED91FC91E9
:1011D0001497EE0FFF1FE00FF11F208931898085E2
:1011E000918501968217930704F5C90101971DC0E7
:1011F000E881F9810284F385E02D60E070E0CE01A2
:1012000009958823A9F0D8011396ED91FC911497C4
:10121000EE0FFF1FE00FF11F808991898F3F91052D
:1012200014F4019602C08FEF90E0918B808B9ECFDB
:10123000E881F9810284F385E02D64E070E0CE015D
:101240000995882381F0D8011396ED91FC911497AC
:10125000EE0FFF1FE00FF11F118610868FE790E061
:10126000918B808B47C0E881F9810284F385E02D62
:101270006BE070E0CE010995882321F0F80114821B
:10128000138223C0E881F9810284F385E02D68E0B0
:1012900070E0CE010995882341F081E090E0D8010B
:1012A00014969C938E93139726C0E881F98102844B
:1012B000F385E02D6AE070E0CE010995882339F0CE
:1012C00082E090E0F8019483838381E051CFE8814C
:1012D000F9810284F385E02D69E070E0CE01099583
:1012E000882309F442C083E090E0D80114969C93CF
:1012F0008E93139781E017968C9337C08091E1020B
:101300009091E202892B61F17801B8E0EB0EF11CBB
:10131000C0E0D0E0F7016081F2E0EF0EF11C8091B7
:10132000E1029091E2028C0F9D1F0E948106809144
:10133000E1029091E2028C0F9D1FD70116966C91ED
:1013400001960E9481062296C830D10519F7809136
:10135000E1029091E202F801638108960E94810601
:10136000D80116961C921E921597DF91CF911F916E
:101370000F91FF90EF90DF90CF9008956F927F9242
:101380008F929F92AF92BF92CF92DF92EF92FF9295
:101390000F931F93CF93DF9300D000D0CDB7DEB76C
:1013A0008C01DC0191968C9191978111E1C088E0CC
:1013B000E8E1F1E01F9601900D928A95E1F7D801DE
:1013C000AE58BF4F80E090E067E070E041E050E051
:1013D0009C0127703327FB01E21BF30B3A0102C08B
:1013E000660C771CEA95E2F79301FC0133E0F59572
:1013F000E7953A95E1F7E00FF11F378523232D9309
:1014000001968034910521F7780162E2E60EF11C25
:1014100080E4D7011D928A95E9F71C8261E0CE0134
:1014200004960E949A106AE070E0C7010E9445117C
:10143000C8018E549F4F2AE0FC0111922A95E9F7CA
:101440004701F70140E050E077E0C72ED12CA19191
:101450009A0163E0359527956A95E1F7200F311FD2
:10146000590162EBA60EB11C61E070E0A11102C04F
:1014700060E070E0DA01A770BB2736016A1A7B0AC8
:1014800001C0660F6A94EAF7D901AE54BF4F2C91A0
:10149000622BD5016C934F5F5F4F40355105B9F614
:1014A000FC01208121110AC0F801ED54FF4F208179
:1014B000211104C031962081222329F081E0D80136
:1014C00091968C9306C04AE050E060E071E00E9483
:1014D000531F8AE0E3EFF1E0D801579601900D9297
:1014E0008A95E1F780E5F70111928A95E9F781E4A1
:1014F000898361E0CE0101960E949A106AE070E053
:10150000C7010E944511019779F58AE0F8017796A5
:10151000DF011D928A95E9F720E030E047E050E0D6
:10152000F40161914F01F90193E0F595E7959A95E2
:10153000E1F7E00FF11F81E090E0611102C080E06F
:1015400090E0B901677077273A01661A770A01C0FF
:10155000880F6A94EAF79789892B878B2F5F3F4F13
:1015600020353105E9F6B8C0D80191961C92B4C077
:10157000D8011896ED91FC9119978281811103C0D1
:10158000EAE0F1E002C0EDE0F1E080819181A2812A
:1015900089839A83AB8363E0CE0101960E949A10FF
:1015A0007801B2E2EB0EF11C68E070E0C7010E9426
:1015B0004511F80182A5882309F48CC020E4F701C5
:1015C000C8018E589F4FDC0101900D922A95E1F7DA
:1015D00028E0F8013F96DF011D922A95E9F7DC012A
:1015E00020E030E047E050E06D91F90183E0F595AF
:1015F000E7958A95E1F7E00FF11F81E090E0611136
:1016000002C080E090E0B901677077273A01661A5E
:10161000770A01C0880F6A94EAF79785892B878734
:101620002F5F3F4F20343105F9F665EF71E0F80187
:1016300020E030E0DB015D91BD01818990E0418DCA
:10164000450F841B910947FD939597FD07C08F3F78
:10165000910529F024F08FEF90E001C080E0818BAC
:10166000A8014E575F4F982F9078DA019C934F5FF7
:101670005F4F982F9074DA019C934F5F5F4F982FC4
:101680009072DA019C934F5F5F4F982F9071DA014F
:101690009C934F5F5F4F982F9870DA019C934F5F38
:1016A0005F4F982F9470DA019C934F5F5F4F982F94
:1016B0009270DA019C934F5F5F4F8170DA018C93D7
:1016C0002F5F3F4F3196085F1F4F2630310509F0DD
:1016D000B1CF02C0F80111A20F900F900F900F90A0
:1016E000DF91CF911F910F91FF90EF90DF90CF90FE
:1016F000BF90AF909F908F907F906F9008950C94C3
:10170000C51E60E070E00C941210EF92FF920F93F0
:101710001F93CF93DF93CDB7DEB728970FB6F8941A
:10172000DEBF0FBECDBF8C01FC01E85BFE4F8081A8
:10173000833440F4813408F075C0882331F080345C
:1017400021F187C08F3F09F084C0FF24F394F09209
:10175000400289E0F8018383148283E0858380E876
:1017600086831782108611861286F386F48640E0FF
:1017700063E0C80103960E945D0FF801F4A660E0E3
:1017800070E0C8010E94121064C08091400288235A
:1017900079F0F0903F02F9E0FF1554F06AE070E054
:1017A00080E090E00E94BB12F394F0923F0237C0B9
:1017B00010923F0280913E0298012C5D3F4F7901CB
:1017C00081110CC028E0C8010396FC01D7010190EB
:1017D0000D922A95E1F741E068E00CC088E0F9013C
:1017E000DE01119601900D928A95E1F741E068E0E3
:1017F000CE0101960E945D0FF801EF2811F41282CC
:1018000007C0E65BFE4F808181708083F801828390
:1018100061E070E0C8010E94121080933E021092B5
:10182000400217C010924002F801138280E88483BE
:1018300085838683878380871186128681E08387EC
:10184000848741E06AE0C80103960E945D0F109210
:101850003F0228960FB6F894DEBF0FBECDBFDF91D2
:10186000CF911F910F91FF90EF900895FC01848D0F
:10187000DF01A80FB11DA35ABF4F2C91848D90E0BA
:1018800001968F739927848FA689B7892C93A08995
:10189000B1898C91837080648C93938D848D98131F
:1018A00006C00288F389E02D80818F7D80830895B2
:1018B000CF92DF92EF92FF920F931F93CF93DF931C
:1018C000EC011A8284E291E0998388831C821B8256
:1018D000198618868FE790E0998B888B1B861A866D
:1018E0009B8B8A8B1D861C869D8B8C8B1F861E86F0
:1018F0009F8B8E8B0091E1021091E2020115110580
:1019000009F05DC082E00E949C0D8C019093E20280
:101910008093E102009779F569E070E082E00E942F
:10192000110D9093E2028093E102892B09F46BC0C0
:1019300000E010E08091E1029091E20260E0800F0F
:10194000911F0E9481068091E1029091E202800F36
:10195000911F6FE701960E9481060E5F1F4F0830AE
:10196000110541F78091E1029091E20260E0089652
:101970000E94810648C008960E94AB1B90E09C83A1
:101980008B837E0188E0E80EF11C6E01E0E1CE0E53
:10199000D11CC8010E94AB1B90E0F7018193919389
:1019A0007F01C80101960E94AB1B90E0F70197836D
:1019B00086830E5F1F4FCE14DF0459F724C0C80181
:1019C00008960E94AB1B90E09C838B837E01F8E01D
:1019D000EF0EF11C6E0180E1C80ED11CC8010E94FF
:1019E000AB1B90E0F701819391937F01C8010196B1
:1019F0000E94AB1B90E0F701978386830E5F1F4F19
:101A0000EC14FD0459F781E090E09E838D83DF9113
:101A1000CF911F910F91FF90EF90DF90CF9008959D
:101A200008958F929F92AF92BF92CF92DF92EF92E2
:101A3000FF920F931F93CF93DF93C82E5B01E0902B
:101A40004202F0904302C0E0D0E00AE010E0EC1661
:101A5000FD060CF462C0C8010E94AB1B98012E5F0A
:101A60003F4F49018F3F21F0EC16FD0609F04CC0B5
:101A7000C4010E94AB1BD82EEC16FD0651F090E07D
:101A80008A159B050CF440C09C2F8D2FE701E92E91
:101A9000F82E6C2DC8010E94810660E0C8010196F5
:101AA0000E9481060D5F1F4FEC16FD06A1F08D2DE3
:101AB00090E00297A816B9068CF47801EA0CFB1C9A
:101AC0006FEFC7010E9481066D2D6A196350C7012F
:101AD00002960E94810621966A2D01C06D2DC401D7
:101AE0000E94810680914202909143028C179D07CB
:101AF00049F0D0934302C09342026C2F81E090E002
:101B00000E948106C8010BC0C4010E94AB1B90E07B
:101B10000396080F191F21969ACF80E090E0DF917D
:101B2000CF911F910F91FF90EF90DF90CF90BF90DA
:101B3000AF909F908F900895DF92EF92FF920F9356
:101B40001F93CF93DF93D82EE0904202F090430290
:101B500000E010E0CAE0D0E00E151F05CCF4CE0185
:101B60000E94AB1BD81209C0CE0101960E94AB1B8C
:101B7000811103C0CE0103960DC0CE0102960E94D2
:101B8000AB1B90E00396C80FD91F0F5F1F4FE4CF28
:101B900080E090E0DF91CF911F910F91FF90EF9047
:101BA000DF9008950F931F93CF93DF93EC018B0188
:101BB0008E819F81009721F00E94C51E1F821E8288
:101BC0008A819B81009711F00E94C51E1B830A83A6
:101BD000DF91CF911F910F9108952F923F924F92D5
:101BE0005F926F927F928F929F92AF92BF92CF92AD
:101BF000DF92EF92FF920F931F93CF93DF93CDB7B6
:101C0000DEB728970FB6F894DEBF0FBECDBF9E8318
:101C10008D836A017B0120E030E040E053E4C7019E
:101C2000B6010E948D1D181654F420E030E040E803
:101C300053E4C701B6010E94C11B6B017C0120E087
:101C400030E0A901C701B6010E942E1C87FF0BC01E
:101C5000F7FAF094F7F8F094812C912C90E8A92EE3
:101C60009FEBB92E13C020E030E0A901C701B601F7
:101C70000E942E1C882339F0812C912C80E8A82EFC
:101C80008FE3B82E03C0812C912C5401ED81FE818D
:101C900027803084B101032C000C880B990B0E9423
:101CA000DD1C2B013C01A70196010E942E1CED8139
:101CB000FE8118160CF4B5C001851285B801012EFD
:101CC000000C880B990B0E94DD1C69837A838B833F
:101CD0009C83A70196010E948D1D18160CF041C02F
:101CE000ED81FE810584F685E02DFA83E983ED819F
:101CF000FE816385748529813A81621B730B072EEF
:101D0000000C880B990B0E94DD1C6D837E838F83F2
:101D10009887A3019201C701B6010E94C11B9B01D4
:101D2000AC016D817E818F8198850E94921D6B012F
:101D30007C01B80162197309072E000C880B990BFE
:101D40000E94DD1C9B01AC01C701B6010E94331C3F
:101D50006B017C01E981FA81BF01FF0F880B990BB0
:101D600040C020E030E04EEF52E4C701B6010E94CF
:101D70002E1C87FF3DC0ED81FE81238434846FE7F4
:101D800070E062197309072E000C880B990B0E94F2
:101D9000DD1C2B013C0129813A814B815C81C7010B
:101DA000B6010E94C11B9B01AC01C301B2010E949C
:101DB000921D6B017C012FE730E0201B310BB90134
:101DC000330F880B990B0E94DD1C9B01AC01C701EE
:101DD000B6010E94331C6B017C01B101330C880BEE
:101DE000990B0E94DD1C9B01AC01C701B60116C016
:101DF00020E030E04EEF52E4C701B6010E94C11B63
:101E000020E030E0A9010E94921D20E030E0A9010D
:101E10000E94331C20E030E04EEF52E40E94C21BCF
:101E200010C065857685072E000C880B990B0E94E3
:101E3000DD1CA70196010E94921DA30192010E9440
:101E4000331CA50194010E94921D6B017C0120E0CE
:101E500030E040E053EC0E942E1C87FD10C020E0D3
:101E600030E04EEF52E4C701B6010E948D1D1816F6
:101E70004CF0C701B6010E94A51CCB0105C080E84B
:101E80009FEF02C08FE790E028960FB6F894DEBF70
:101E90000FBECDBFDF91CF911F910F91FF90EF90BB
:101EA000DF90CF90BF90AF909F908F907F906F907A
:101EB0005F904F903F902F900895FC0128E0539A37
:101EC000808190E0880F892F881F990B892B09F456
:101ED00030C0000000000000000000000000000012
:101EE0000000539800000000000000000000000007
:101EF00000000000000000000000000000000000E2
:101F000000000000000000000000000000000000D1
:101F100000000000000000000000000000000000C1
:101F200000000000000000000000000000000000B1
:101F300030C00000000000000000000000000000B1
:101F40000000000000000000000000000000000091
:101F50000000000000000000000000000000000081
:101F60000000000000000000000000000000000071
:101F70000000000000000000000000000000000061
:101F80000000000000000000000000000000000051
:101F90005398215069F0000000000000000000008C
:101FA00000000000000000008081880F808387CF40
:101FB0000000000000000000615031F0000000004F
:101FC0000000000031967ACF000000000000000001
:101FD0000000000000000000539A00000000000014
:101FE00000000000000000000000000000000000F1
:101FF0000000000000000000442391F000000000F9
:1020000000000000000000000000000000000000D0
:1020100000000000000000000000000000000000C0
:1020200053980895CF93DF93DC01FC01E85BFE4FEA
:1020300083E0EF0119928A95E9F7EF01161617066A
:102040009CF484EC99E04B9907C081E09C968C93BA
:102050009C9728E030E01BC00197A9F79C968C91D3
:102060009C97882309F461C09C968C919C97811160
:102070000AC080E290E04B9902C080E290E00197B4
:1020800018161906C4F328E030E04B99FECF000083
:102090000000000000000000000000000000000040
:1020A0000000000000000000000000000000000030
:1020B0000000000000000000000000000000000020
:1020C0000000000000000000000000000000000010
:1020D000000000000000000000004B9B03C0808156
:1020E000816080832150310931F08081880F8083A5
:1020F0004B9BFECFCACF8881803441F4CD01865BF3
:102100009E4FE817F90711F03196BDCF4B9BFECFDC
:102110008CE090E04B9902C08CE090E0019718169B
:102120001906C4F381E090E002C080E090E0DF9106
:10213000CF910895FC0128E08AB180638AB980813B
:1021400090E0880F892F881F990B892B09F432C0E2
:10215000000000000000000000000000000000007F
:102160008AB18F7C8AB900000000000000000000E6
:10217000000000000000000000000000000000005F
:10218000000000000000000000000000000000004F
:10219000000000000000000000000000000000003F
:1021A000000000000000000000000000000000002F
:1021B000000032C00000000000000000000000002D
:1021C000000000000000000000000000000000000F
:1021D00000000000000000000000000000000000FF
:1021E00000000000000000000000000000000000EF
:1021F00000000000000000000000000000000000DF
:1022000000000000000000000000000000000000CE
:1022100000008AB18F7C8AB9215069F0000000006B
:1022200000000000000000000000000000008081AD
:10223000880F808381CF0000000000000000615003
:1022400031F00000000000000000319674CF000063
:1022500000000000000000000000000000008AB143
:1022600080638AB900000000000000000000000048
:10227000000000000000000000000000000000005E
:1022800000008AB18F7C8AB90895FC01660F660F41
:10229000660F9FE329B1207329F09150D9F780E0B0
:1022A00090E0089500000000000000000000000021
:1022B000000000000000000000000000000000001E
:1022C000000000000000000000000000000000000E
:1022D00000000000000000000000000000000000FE
:1022E00000000000000000000000000000000000EE
:1022F00099B190739193615051F09FE329B120738C
:1023000009F0C7CF9150D1F782E090E0089581E0C5
:1023100090E008954F925F926F927F928F929F927A
:10232000AF92BF92CF92DF92EF92FF92CF93DF9363
:10233000EC016A017B0120E030E040E053E4C7019A
:10234000B6010E948D1D181654F420E030E040E8DC
:1023500053E4C701B6010E94C11B6B017C0120E060
:1023600030E0A901C701B6010E942E1C87FF0BC0F7
:10237000F7FAF094F7F8F094812C912C40E8A42E11
:102380004FEBB42E13C020E030E0A901C701B60125
:102390000E942E1C882339F0812C912C30E8A32E2A
:1023A0003FE3B32E03C0812C912C54018B819C817F
:1023B000880F991FC80FD91F68857985072E000CD3
:1023C000880B990B0E94DD1C2B013C01A701960193
:1023D0000E948D1D87FF44C0A3019201C701B60171
:1023E0000E94C11B6B017C01A301920160E070E0BF
:1023F0008EEF92E40E94C11B9B01AC01C701B601A4
:102400000E94331C6B017C0168897989072E000CBE
:10241000880B990B0E94DD1C9B01AC01C701B60122
:102420000E94921DA50194010E94921D6B017C01E6
:1024300020E030E040E053EC0E942E1C87FD13C0EA
:1024400020E030E04EEF52E4C701B6010E948D1D3E
:10245000181664F0C701B6010E94A51CCB0108C084
:1024600080E090E005C080E89FEF02C08FE790E039
:10247000DF91CF91FF90EF90DF90CF90BF90AF9022
:102480009F908F907F906F905F904F900895CF9323
:10249000DF9390E0FC01EC55FF4F2491FC01E057E5
:1024A000FF4F84918823C1F090E0880F991FFC01B1
:1024B000EA57FF4FC591D491FC01E458FF4FA59115
:1024C000B4919FB7F8948881E22FE0958E2388839A
:1024D0008C91E823EC939FBFDF91CF91089590E01A
:1024E000FC01E859FF4F2491FC01EC55FF4F34915A
:1024F000FC01E057FF4FE491EE23B9F1222339F1BB
:10250000233091F038F42130A9F0223001F584B560
:102510008F7D12C0273091F02830A1F02430B9F41B
:10252000809180008F7D03C0809180008F778093A1
:1025300080000DC084B58F7784BD09C08091B00044
:102540008F7703C08091B0008F7D8093B000F0E062
:10255000EE0FFF1FE458FF4FA591B4919FB7F89479
:102560008C91309538233C939FBF0895682F84E465
:1025700092E00C946A178F929F92AF92BF92CF9283
:10258000DF92EF92FF926B017C010E94D9174B0101
:102590005C01C114D104E104F104F1F00E94D917E7
:1025A000DC01CB0188199909AA09BB09883E93402F
:1025B000A105B10570F321E0C21AD108E108F108C4
:1025C00088EE880E83E0981EA11CB11CC114D104B2
:1025D000E104F10419F7DDCFFF90EF90DF90CF9089
:1025E000BF90AF909F908F9008952091E502309119
:1025F000E6022115310529F0682FC90101960C94D6
:1026000081060895682F8091E5029091E602009777
:1026100011F00C9481060895DF92EF92FF920F93D0
:102620001F93CF93DF93EC018B017A018C819D8105
:102630008130910521F0029709F471C011C0DB01CE
:10264000ED91FC910088F189E02DCB01099588235B
:1026500029F082E090E09D838C83DDC11D821C8285
:10266000D801ED91FC910680F781E02D60E070E0EB
:10267000C8010995D801ED91FC910084F185E02D08
:1026800060E070E0C8010995D801ED91FC910680E9
:10269000F781E02D60E070E0C8010995682F880F90
:1026A000770B880B990B0E94DD1CAB01BC01CE019E
:1026B0000E94ED0DD82ED801ED91FC910084F1859A
:1026C000E02D60E070E0C8010995682F880F770B56
:1026D000880B990B0E94DD1CAB01BC01CE010E944E
:1026E000ED0DC82FD701ED91FC910284F385E02D0B
:1026F0004D2D60E070E0C7010995D701ED91FC9187
:102700000484F585E02D4C2F60E070E0C701DF9177
:10271000CF911F910F91FF90EF90DF900994AF81BF
:10272000B885A25CBE4FFA0180819181FC012285AF
:1027300033854C9160E070E0C701F9010995A985E6
:10274000BA85A25CBE4FF70180819181FC0124858E
:1027500035854C9160E070E0C701F9010995D80119
:10276000ED91FC910088F189E02DC801099588233D
:1027700009F454C18E81D801ED91FC910284F38556
:10278000E02D882309F468C062E070E0C801099573
:1027900081115FC1D801ED91FC910284F385E02D98
:1027A00063E070E0C8010995811153C1D801ED9132
:1027B000FC910284F385E02D61E070E0C801099589
:1027C000811147C1D801ED91FC910284F385E02D80
:1027D00060E070E0C801099581113BC1D801ED911D
:1027E000FC910284F385E02D68E070E0C801099552
:1027F00081112FC1D801ED91FC910284F385E02D68
:1028000069E070E0C8010995811123C1D801ED91FB
:10281000FC910284F385E02D6AE070E0C80109951F
:10282000811117C1D801ED91FC910284F385E02D4F
:102830006CE070E0C801099581110BC1D801ED91E0
:10284000FC910284F385E02D64E070E0C8010995F5
:102850008111FFC01E82FDC063E070E0C8010995D0
:10286000882351F08F8198858230910514F001976B
:1028700019C081E090E016C0D801ED91FC9102846E
:10288000F385E02D62E070E0C8010995882369F0C6
:102890002F81388589859A8501972817390714F47F
:1028A000C901019698878F83B6C0D801ED91FC913C
:1028B0000284F385E02D61E070E0C801099588236A
:1028C00061F029853A858F81988501968217930753
:1028D0000CF051C0C90101974EC0D801ED91FC9197
:1028E0000284F385E02D60E070E0C801099588233B
:1028F00051F089859A858E37910514F401963BC075
:102900008EE790E038C0D801ED91FC910284F38508
:10291000E02D64E070E0C80109958823D1F08B8137
:10292000813049F0823071F087E190E098878F83A1
:1029300085E290E020C084E190E098878F8380E278
:1029400090E019C08EE190E098878F8389E290E053
:1029500012C0D801ED91FC910284F385E02D6CE06A
:1029600070E0C8010995882349F088E090E09887D5
:102970008F838AE290E09A8789874DC0D801ED91D4
:10298000FC910284F385E02D68E070E0C8010995B0
:10299000882369F082E08B838EE190E09E878D87AB
:1029A00089E290E09C878B8789E490E032C0D8016F
:1029B000ED91FC910284F385E02D6AE070E0C8019E
:1029C0000995882379F081E08B8324E130E03E870C
:1029D0002D8720E230E03C872B8725E330E0388BE1
:1029E0002F871AC0D801ED91FC910284F385E02D68
:1029F00069E070E0C8010995882359F11B8287E1DD
:102A000090E09E878D8785E290E09C878B8787E4A6
:102A100090E0988B8F8781E08E831BC08091E302CA
:102A20009091E402009799F06F810E948106809155
:102A3000E3029091E402698501960E9481068091EB
:102A4000E3029091E4026B8102960E9481061D824E
:102A50001C82DF91CF911F910F91FF90EF90DF903B
:102A600008950F931F93CF93DF93EC011A828CE3A9
:102A700091E0998388831B820091E3021091E40224
:102A800001151105F1F581E00E949C0D8C019093D8
:102A9000E4028093E302892BA1F563E070E081E01A
:102AA0000E94110D9093E4028093E3021B8227E1C0
:102AB00030E03E872D8725E230E03C872B8727E4F6
:102AC00030E0388B2F8728E030E038872F832AE2E8
:102AD00030E03A872987009731F168E00E9481064B
:102AE0008091E3029091E402698501960E9481063B
:102AF0008091E3029091E4026B8102960E9481062C
:102B000012C0C8010E94AB1B90E098878F83C80158
:102B100001960E94AB1B90E09A878987C8010296B4
:102B20000E94AB1B8B838B81813069F08230B1F0C6
:102B300087E190E09E878D8785E290E09C878B8778
:102B400087E490E015C084E190E09E878D8780E265
:102B500090E09C878B8785E390E00AC08EE190E04F
:102B60009E878D8789E290E09C878B8789E490E03F
:102B7000988B8F8789859A858038910524F08EE718
:102B800090E09A87898789859A852F813885821771
:102B900093071CF4019798878F8381E090E09D83D1
:102BA0008C83DF91CF911F910F9108958091E50261
:102BB0009091E602892BF9F480E00E949C0D90939D
:102BC000E6028093E502892BB1F462E070E080E0D8
:102BD0000E94110D9093E6028093E502009759F050
:102BE00061E00E9481068091E5029091E60260E03A
:102BF00001960C94810608950F931F93CF93DF9352
:102C00008C01EB01FC018381E881F981882359F073
:102C10000684F785E02DCB010995882309F4EAC0E5
:102C2000F8011382E7C00284F385E02D64E070E0D0
:102C3000CE010995882381F083E090E00E942D1E4B
:102C4000FC0112822FE232E031832083BC01CE01ED
:102C50000E94D20D80E017C0E881F9810284F385DB
:102C6000E02D61E070E0CE010995882391F081E1CB
:102C700090E00E942D1E8C010E943115B801CE01FA
:102C80000E94D20D81E0DF91CF911F910F910C94A2
:102C90000213E881F9810284F385E02D6EE070E093
:102CA000CE0109958823D1F082E090E00E942D1E8C
:102CB0008C0187E192E0F801918380838C819D8172
:102CC000009711F00E94C51E1D830C838E819F8189
:102CD0009B838A831F821E8280E086C0E881F981FF
:102CE0000284F385E02D63E070E0CE01099588232E
:102CF00069F088E190E00E942D1E8C010E94580C22
:102D0000B801CE010E94D20D82E0BDCFE881F981E9
:102D10000284F385E02D69E070E0CE0109958823F7
:102D2000D1F082E090E00E942D1E8C0189E292E0B9
:102D3000F801918380838C819D81009711F00E941E
:102D4000C51E1D830C838E819F819B838A831F8276
:102D50001E8281E049C0E881F9810284F385E02D7B
:102D60006AE070E0CE0109958823D1F082E090E01E
:102D70000E942D1E8C0183E292E0F80191838083F2
:102D80008C819D81009711F00E94C51E1D830C83CC
:102D90008E819F819B838A831F821E8282E024C052
:102DA000E881F9810284F385E02D6BE070E0CE01CB
:102DB00009958823F9F082E090E00E942D1E8C0195
:102DC0008DE192E0F801918380838C819D81009751
:102DD00011F00E94C51E1D830C838E819F819B83F1
:102DE0008A831F821E8283E0DF91CF911F910F9112
:102DF0000C94F512DF91CF911F910F910895CF920E
:102E0000DF92EF92FF920F931F93CF93DF936C01AA
:102E10007A018B01C0E0D0E0CE15DF0581F0D8014A
:102E20006D918D01D601ED91FC910190F081E02D25
:102E3000C6010995892B11F02196EECF7E01C701BD
:102E4000DF91CF911F910F91FF90EF90DF90CF9086
:102E50000895089580E090E00895FC01538D448D1D
:102E6000252F30E0842F90E0821B930B541710F035
:102E7000CF96089501970895FC01918D828D981742
:102E800061F0828DDF01A80FB11D5D968C91928D4E
:102E90009F5F9F73928F90E008958FEF9FEF08954B
:102EA000FC01918D828D981731F0828DE80FF11D14
:102EB000858D90E008958FEF9FEF08950E944E1F3B
:102EC00084E492E00E94930621E0892B09F420E03B
:102ED000822F0895EF92FF920F931F93CF93DF936A
:102EE000EC0181E0888F9B8D8C8D981305C0E8895B
:102EF000F989808185FD26C0F62E0B8D10E00F5FCD
:102F00001F4F0F731127E02E8C8DE8120CC00FB6E7
:102F100007FCFACFE889F989808185FFF5CFCE01DA
:102F20000E94360CF1CF8B8DFE01E80FF11DE35AA4
:102F3000FF4FF0829FB7F8940B8FEA89FB8980815D
:102F400080620AC09FB7F894EE89FF896083E889A0
:102F5000F98980818370806480839FBF81E090E0E5
:102F6000DF91CF911F910F91FF90EF900895CF9334
:102F7000DF93EC01888D8823C9F0EA89FB89808181
:102F800085FD05C0A889B9898C9186FD0FC00FB653
:102F900007FCF5CF808185FFF2CFA889B9898C9194
:102FA00085FFEDCFCE010E94360CE7CFDF91CF91A8
:102FB00008953FB7F8948091F1029091F202A091A8
:102FC000F302B091F40226B5A89B05C02F3F19F07B
:102FD0000196A11DB11D3FBFBA2FA92F982F882799
:102FE000820F911DA11DB11DBC01CD0142E0660FF4
:102FF000771F881F991F4A95D1F708951F920F9246
:103000000FB60F9211242F933F938F939F93AF93FB
:10301000BF938091ED029091EE02A091EF02B091EA
:10302000F0023091EC0223E0230F2D3720F40196BB
:10303000A11DB11D05C026E8230F0296A11DB11DDB
:103040002093EC028093ED029093EE02A093EF02A6
:10305000B093F0028091F1029091F202A091F302FC
:10306000B091F4020196A11DB11D8093F1029093DD
:10307000F202A093F302B093F402BF91AF919F913B
:103080008F913F912F910F900FBE0F901F90189529
:103090001F920F920FB60F9211242F933F934F93CD
:1030A0005F936F937F938F939F93AF93BF93EF93B0
:1030B000FF9384E492E00E94360CFF91EF91BF9160
:1030C000AF919F918F917F916F915F914F913F91C0
:1030D0002F910F900FBE0F901F9018951F920F9277
:1030E0000FB60F9211242F938F939F93EF93FF931B
:1030F000E0915402F09155028081E0915A02F091E2
:103100005B0282FD12C0908180915D028F5F8F73A0
:1031100020915E02821751F0E0915D02F0E0EC5BDD
:10312000FD4F958F80935D0201C08081FF91EF91EB
:103130009F918F912F910F900FBE0F901F90189518
:10314000E4E4F2E01382128288EE93E0A0E0B0E0C3
:1031500084839583A683B7838AE291E091838083F9
:1031600085EC90E09587848784EC90E0978786874C
:1031700080EC90E0918B808B81EC90E0938B828B44
:1031800082EC90E0958B848B86EC90E0978B868B1D
:10319000118E128E138E148E1092E2021092E102A2
:1031A0001092E4021092E3021092E6021092E502FD
:1031B0000895CF93DF9300D01F92CDB7DEB77894F8
:1031C00084B5826084BD84B5816084BD85B582602C
:1031D00085BD85B5816085BD80916E0081608093DD
:1031E0006E00109281008091810082608093810046
:1031F0008091810081608093810080918000816056
:10320000809380008091B10084608093B1008091B0
:10321000B00081608093B00080917A0084608093D8
:103220007A0080917A00826080937A0080917A009F
:10323000816080937A0080917A00806880937A0020
:103240001092C100E0915402F091550282E0808317
:10325000E0915002F09151021082E0915202F091FF
:10326000530280E1808310925C02E0915802F09159
:10327000590286E08083E0915602F09157028081E6
:1032800080618083E0915602F091570280818860CE
:103290008083E0915602F09157028081806880839C
:1032A000E0915602F091570280818F7D808380915A
:1032B00010019091110101979093110180931001D9
:1032C00043E050E062E070E0CE0101960E949B1B5B
:1032D0008981853A31F48A818E3919F48B818C3851
:1032E00011F080E04DC089E090E00E94AB1B82337A
:1032F000A1F162E389E090E00E948106109243020E
:103300001092420260E080E090E00E9481066091AD
:10331000420281E090E00E9481068091BE0190917E
:10332000BF01A091C00189839A83AB83CE0101962E
:103330007C0102E010E0D701DD907D01C8010E9410
:10334000AB1BD81621F06D2DC8010E94B31B0F5F77
:103350001F4F0530110579F712C080E090E00E9400
:10336000AB1B90E0909343028093420281E090E097
:103370000E94AB1B90E0909343028093420281E055
:103380008093EB028BE491E00E942D1E8C0185EC72
:1033900091E0F80191838083339681E2DF011D92F1
:1033A0008A95E9F7EB5BFE4F83E0DF011D928A957A
:1033B000E9F7F80114A61093EA020093E9028CEBF6
:1033C00090E00E942D1E21E032E0DC0111963C933A
:1033D0002E939C012E583F4F1D963C932E931C9785
:1033E00020E430E01B963C932E931A971E961C9275
:1033F0001E9791961C9291972AE0E3EFF1E0579681
:1034000001900D922A95E1F79093E8028093E702EC
:1034100083E00E946F1283E00E944712F80112823B
:103420000E94D6158091E5029091E602009749F03E
:1034300001960E94AB1B823091F08330D1F0813035
:1034400039F082E090E00E942D1E27E132E00DC0AD
:1034500082E090E00E942D1E29E232E010C082E05E
:1034600090E00E942D1E23E232E0DC012D933C937C
:1034700009C082E090E00E942D1E2DE132E0FC01A7
:10348000318320836C010E94D6158091E5029091D2
:10349000E602009731F00E94AB1B813081F0823050
:1034A000B1F083E090E00E942D1EDC0112961C9288
:1034B00012972FE232E02D933C938C010FC081E1F3
:1034C00090E00E942D1E8C010E94311507C088E1FA
:1034D00090E00E942D1E8C010E94580CA090E902E1
:1034E000B090EA02E090E702F090E80285E00E94E6
:1034F0006F1285E00E94471284E00E946F1284E000
:103500000E944712F701B186A08602831383C4820A
:10351000D5821782168235E3632E32E0732E55244E
:10352000539448E0842E912C8091EB02882309F477
:10353000F7C08091E9029091EA02DC01ED91FC91E3
:103540000190F081E02D09958111D2C00091E70230
:103550001091E802F8018685C484D584A284B384DE
:10356000882351F1E12CF12CEA14FB0464F5C70126
:10357000F7FC079623E0959587952A95E1F7F601E4
:10358000E80FF91F2081022E000C330BC701B40194
:103590000E94FF1D02C0359527958A95E2F7C90163
:1035A0008170992720FF02C081E390E00E94B6124B
:1035B000FFEFEF1AFF0AD8CF7601C7018C199D09DA
:1035C0008A159B057CF08AE090E00E94B612D80133
:1035D000ED91FC910484F585E02DC80109958111D8
:1035E0000EC038C0F70181917F01882319F081E373
:1035F00090E002C080E090E00E94B612DECFD801D9
:103600001296ED91FC911397309719F082818111F8
:1036100021C084E090E00E942D1E7C01FC0171829B
:10362000608253825282892B09F47DC0F801868121
:103630009781009711F00E94C51ED80112968D91B6
:103640009C91139717969C938E9316971396FC92C2
:10365000EE9212976091100170911101072E000CEB
:10366000880B990B0E94BB12F8940091E70210910D
:10367000E802D801ED91FC910480F581E02DC801AC
:103680000995F80180859185DC01ED91FC9100841C
:10369000F185E02D0995F80182819381009751F021
:1036A00040855185DC01ED91FC910190F081E02D88
:1036B000B8010995F80186819781892B71F484817D
:1036C0009581009751F040855185DC01ED91FC9189
:1036D0000190F081E02DB80109958091E902909167
:1036E000EA02DC01ED91FC910480F581E02D099561
:1036F0008091E9029091EA02DC01ED91FC91028057
:10370000F381E02D0995F8948091E9029091EA0205
:10371000DC01ED91FC910680F781E02D099578940C
:103720000E949F0601CFF80186819781938382834F
:10373000178216828FCFDC01CB01FC01F999FECFF5
:1037400006C0F2BDE1BDF89A319600B40D92415029
:103750005040B8F70895F999FECF92BD81BDF89A0F
:10376000992780B50895262FF999FECF1FBA92BDEB
:1037700081BD20BD0FB6F894FA9AF99A0FBE019652
:1037800008955058BB27AA270E94D91B0C94531D9B
:103790000E94451D38F00E944C1D20F039F49F3FD7
:1037A00019F426F40C94421D0EF4E095E7FB0C94FA
:1037B0003C1DE92F0E94641D58F3BA176207730776
:1037C0008407950720F079F4A6F50C94861D0EF475
:1037D000E0950B2EBA2FA02D0B01B90190010C0121
:1037E000CA01A0011124FF27591B99F0593F50F439
:1037F000503E68F11A16F040A22F232F342F442791
:10380000585FF3CF469537952795A795F040539588
:10381000C9F77EF41F16BA0B620B730B840BBAF058
:103820009150A1F0FF0FBB1F661F771F881FC2F7C3
:103830000EC0BA0F621F731F841F48F487957795D7
:103840006795B795F7959E3F08F0B0CF9395880F91
:1038500008F09927EE0F9795879508950E94181DF7
:1038600008F481E008950E94471C0C94531D0E94A7
:103870004C1D58F00E94451D40F029F45F3F29F08F
:103880000C943C1D51110C94871D0C94421D0E94F8
:10389000641D68F39923B1F3552391F3951B550BE0
:1038A000BB27AA2762177307840738F09F5F5F4F13
:1038B000220F331F441FAA1FA9F335D00E2E3AF052
:1038C000E0E832D091505040E695001CCAF72BD06A
:1038D000FE2F29D0660F771F881FBB1F26173707BB
:1038E0004807AB07B0E809F0BB0B802DBF01FF27ED
:1038F00093585F4F3AF09E3F510578F00C943C1D71
:103900000C94871D5F3FE4F3983ED4F3869577953A
:103910006795B795F7959F5FC9F7880F911D9695A5
:10392000879597F90895E1E0660F771F881FBB1F01
:10393000621773078407BA0720F0621B730B840BAE
:10394000BA0BEE1F88F7E09508950E94AC1C6894AE
:10395000B1110C94871D08950E946C1D88F09F572B
:1039600098F0B92F9927B751B0F0E1F0660F771FA3
:10397000881F991F1AF0BA95C9F714C0B13091F099
:103980000E94861DB1E008950C94861D672F782F44
:103990008827B85F39F0B93FCCF38695779567955E
:1039A000B395D9F73EF490958095709561957F4FCA
:1039B0008F4F9F4F0895E89409C097FB3EF4909570
:1039C0008095709561957F4F8F4F9F4F9923A9F0F8
:1039D000F92F96E9BB279395F69587957795679587
:1039E000B795F111F8CFFAF4BB0F11F460FF1BC0CB
:1039F0006F5F7F4F8F4F9F4F16C0882311F096E95E
:103A000011C0772321F09EE8872F762F05C066230B
:103A100071F096E8862F70E060E02AF09A95660FC4
:103A2000771F881FDAF7880F9695879597F908957D
:103A3000990F0008550FAA0BE0E8FEEF16161706BF
:103A4000E807F907C0F012161306E407F50798F027
:103A5000621B730B840B950B39F40A2661F0232B40
:103A6000242B252B21F408950A2609F4A140A695BC
:103A70008FEF811D811D089597F99F6780E870E0A1
:103A800060E008959FEF80EC089500240A941616D4
:103A9000170618060906089500240A94121613063C
:103AA000140605060895092E0394000C11F48823CA
:103AB00052F0BB0F40F4BF2B11F460FF04C06F5FE6
:103AC0007F4F8F4F9F4F089557FD9058440F551FBC
:103AD00059F05F3F71F04795880F97FB991F61F090
:103AE0009F3F79F087950895121613061406551F07
:103AF000F2CF4695F1DF08C0161617061806991F73
:103B0000F1CF86957105610508940895E894BB2767
:103B100066277727CB0197F908950E94181D08F4AE
:103B20008FEF08950E94A51D0C94531D0E94451D02
:103B300038F00E944C1D20F0952311F00C943C1D90
:103B40000C94421D11240C94871D0E94641D70F377
:103B5000959FC1F3950F50E0551F629FF001729F32
:103B6000BB27F00DB11D639FAA27F00DB11DAA1F41
:103B7000649F6627B00DA11D661F829F2227B00D8E
:103B8000A11D621F739FB00DA11D621F839FA00D19
:103B9000611D221F749F3327A00D611D231F849F69
:103BA000600D211D822F762F6A2F11249F575040C0
:103BB0009AF0F1F088234AF0EE0FFF1FBB1F661F3B
:103BC000771F881F91505040A9F79E3F510580F004
:103BD0000C943C1D0C94871D5F3FE4F3983ED4F396
:103BE000869577956795B795F795E7959F5FC1F7A8
:103BF000FE2B880F911D9695879597F9089597FB51
:103C0000072E16F4009407D077FD09D00E94131EEA
:103C100007FC05D03EF4909581959F4F08957095CF
:103C200061957F4F0895AA1BBB1B51E107C0AA1FD6
:103C3000BB1FA617B70710F0A61BB70B881F991F4D
:103C40005A95A9F780959095BC01CD010895EE0F86
:103C5000FF1F0590F491E02D09940F931F93CF93CC
:103C6000DF938230910510F482E090E0E091F7025A
:103C7000F091F80220E030E0A0E0B0E0309719F1D8
:103C8000408151810281138148175907C8F0841778
:103C9000950769F4109731F012960C9312971396CA
:103CA0001C9327C00093F7021093F80222C021153D
:103CB000310519F04217530718F49A01BD01EF01BD
:103CC000DF01F801DBCF21153105F9F0281B390B95
:103CD0002430310580F48A819B816115710521F0C2
:103CE000FB019383828304C09093F8028093F702D0
:103CF000FE01329644C0FE01E20FF31F81939193BF
:103D000022503109398328833AC02091F50230913D
:103D1000F602232B41F420911401309115013093C8
:103D2000F6022093F5022091120130911301211522
:103D3000310541F42DB73EB740911601509117015E
:103D4000241B350BE091F502F091F602E217F30720
:103D5000A0F42E1B3F0B2817390778F0AC014E5FFB
:103D60005F4F2417350748F04E0F5F1F5093F60240
:103D70004093F5028193919302C0E0E0F0E0CF011F
:103D8000DF91CF911F910F910895CF93DF9300970B
:103D900009F481C0FC01329713821282A091F702CC
:103DA000B091F802109781F420813181820F931F26
:103DB0002091F5023091F6022817390751F5F0935A
:103DC000F602E093F50267C0ED0120E030E0CE1787
:103DD000DF0740F44A815B819E0141155105F1F0F6
:103DE000EA01F5CFD383C28340815181840F951FAF
:103DF000C817D90759F488819981840F951F0296B5
:103E0000918380838A819B819383828321153105ED
:103E100029F4F093F802E093F7023DC0E901FB8337
:103E2000EA8349915991C40FD51FEC17FD0761F43E
:103E300080819181840F951F0296E901998388837F
:103E4000828193819B838A83E0E0F0E012968D91DA
:103E50009C911397009719F0FD01DC01F7CF8D912C
:103E60009C9111979D012E5F3F4F820F931F2091D0
:103E7000F5023091F6022817390769F4309729F4D2
:103E80001092F8021092F70202C013821282B093CD
:103E9000F602A093F502DF91CF91089581E090E0C2
:103EA000F8940C945A1FDC0101C06D9341505040AE
:083EB000E0F70895F894FFCF3C
:103EB8000900030000000000010140030040030165
:103EC8000C000000F902800000807F7F7F7F0000E7
:103ED800000000007C07000000006A17FF162D177D
:103EE800B71793063C175017000000000C1300107A
:103EF800111213141516171718191A1B1B1C1D1E3F
:103F08001E1F20212222232424252626272828296B
:103F18002A2A2B2C2C2D2D2E2F2F303031313233B5
:103F280033343435353636373738383839393A3A1C
:103F38003B3B3B3C3C3D3D3D3E3E3F3F3F404040A0
:103F48004041414142424243434343434444444441
:103F58004445454545454646464646464646464600
:103F68004747474747474747474747474747A59E24
:103F78008C00000000F806F506810B850B710767B9
:103F8800075F07510745070107FB06060700000002
:103F980000000000005E175E175E175E175E175E72
:103FA800175E1700808080808000000202000000F9
:103FB80000100D7F0BBE09ED06E506C806BC06B26B
:103FC80006A9060000000023030000000087000087
:103FD800000000D50100000000A7040000000071E7
:0E3FE8000400000000FC15000000005E170041
:00000001FF
